:0600000061C0FECFD9C073
:10000600FCCFFBCF91C0F9CFDAC0F7CFF6CFF5CF53
:10001600F4CFF3CF83C0F1CFF0CFEFCFEECFEDCF5C
:10002600ECCFEBCF1027E80364000A0001000010B4
:100036000001100001000000000024504D544B3315
:1000460031342C302C312C302C312C312C352C30B9
:100056002C302C302C302C302C302C302C302C30BA
:100066002C302C302C302C302A32430D0A002450F0
:100076004D544B3330312C302A32430D0A00245074
:100086004D544B3836392C312C302A33340D0A0076
:1000960024504D544B3235312C31343430302A32E1
:1000A600390D0A0024504D544B3232302C35303045
:1000B6002A32420D0A00040008003C000000F894B1
:1000C600EE27ECBBE5BFF8E1A895A4B7A77FA4BFD0
:1000D600F1BDE1BD8DE0A2E0ED938A95E9F780E8F8
:1000E600A0E6ED938A95E9F7ECEBF0E08591959122
:1000F600009761F0A591B59105901590BF01F001AB
:1001060005900D920197E1F7FB01F0CFE0E0E3BB2C
:10011600E4BBE5BBEFEDEDBFC0E872C1EA9398988A
:10012600E0E0E0BFE3BF49C0AA93EA93EFB7EA93E2
:1001360057D2A0E09999A1E0E1E0EA2711F4999855
:1001460001C0999A9F9B03C09F98E0E8EBBFC098B7
:10015600849B06C03394E5E0E31511F494983324A8
:10016600859B16C094982394E5E0E21589F4A0E0F7
:100176009A99A1E0E1E0EA2711F49A9801C09A9AC7
:100186002224E1E0E71520F0E71509F49B9A739421
:100196009B9B02C09C9901C007C05394E8E0E515FB
:1001A60019F49C9844245524E991EFBFE991A9914B
:1001B6001895EA939E9AE0E0EBBFE9911895EA93C9
:1001C600EFB7EA9375D21BB10CB1E12FEC7171F464
:1001D600E92D9394E0580083E8E0E91509F49924A1
:1001E600B394E8E0EB1511F4BB24A09A0991199198
:1001F600E991EFBFE99118951A93989AE2E0E0BF6A
:10020600E3E0E3BFE0E0E2BFE5EEE6BFE5E0E8BF3E
:10021600BB2011F4989901C001C0FACF989B0CC07D
:10022600E82D8394E0581081E8E0E81509F4882465
:10023600F894BA947894E12F19910895BA93AA93F1
:100246001A9310E0EB811E1750F4969AA981BA8191
:1002560018D29698A981BA8114D21F5FF3CF18815C
:1002660067C1BA93AA9324D200E010E0C498EB8148
:10027600F070BBD1FE2FE0E08F01EA81B6D1F0E04D
:100286000E2B1F2BC49AF80118D252C1AA93829939
:10029600FECFE881EFB9CCD1CBD1CAD1C9D1C8D173
:1002A600C7D1C6D1C5D185C1A0E0BEEFDADFA6E9C8
:1002B600C4D1A8EDB0E8D5DFA0E2B6EAD2DFA5E06A
:1002C600B6ECCFDFA0EAB4E9CCDFACEEB2ECC9DF26
:1002D600A3E8BAECC6DFA6EDBEECC3DFABE9B4EC2F
:1002E600C0DFA5E5B8E9BDDFA7E7BCECBADFA0E053
:1002F600B0EEB7DFA0E0B8ECB4DFA0E0B0ECD3C05E
:10030600FF921A93E1E0FE2E10E0F0FE43C0239721
:1003160073DFEA83AA81A432B1F46EDFE9836CDF6E
:10032600E883A981A73419F4A881A03509F00BC088
:10033600F1FC0FC0E894F0F8E3E0EA93A4E6B0E03D
:100346007DDF239627C0123511F5EFE5E9B9A4E65E
:1003560074D1F894A0E4B0E02ED1A4E7B0E02BD19C
:10036600A4E8B0E028D1A6E9B0E025D1A4E665D19D
:10037600EFE3E9B9A4EFB1E084D1AAEAB0E01BD17A
:10038600E1E05DD1E894F1F810E0789401C01F5FD8
:100396002396BBCF1991FF900895E0E8E6BDE0E013
:1003A600E6BDE4E0EBBBE0E0EABBE5EDE7BBE4E19C
:1003B600E8BBE2E5E1BBEDE2E2BBE0E0EFBDE4E095
:1003C600EEBD0ED1E0E0E5BDE4BDEBBDEABDE9BDA5
:1003D600E8BDE1E8E9BFE0E0E5BFE0E8EBBFEABF82
:1003E600E0E0EDB9EBB9E8E9EAB9E6E0E3B9E0E067
:1003F600E2B9EFE3E9B9E0E8E8B9E0E0E1B9089588
:10040600CCDF78947DDFF8944FDFE2E018D1789462
:100416001AD1C2988FD09899FDCF9B9B02C09C9B06
:1004260001C005C04394E6E0E41509F49C9ABB209C
:1004360029F09B9B02C09C9901C008C09E9B04C0EA
:10044600A1E090D09E989F9A30D0F1CFE1CFFFCF18
:10045600B39B23C0989AE2E0E0BFE3E0E3BFE0E0AD
:10046600E2BFE5EEE6BFE5E0E8BFB19902C09899C4
:1004760001C001C0FACFB39B02C0B19901C00DC043
:10048600C698C298C498D4D0D3D0D2D0D1D0D0D028
:10049600CFD0CED0CDD0EFB108950895A1E8BAEC73
:1004A600E0DEA3E8BAECDDDE089500D1D0D0F6DFB9
:1004B600A0E0B0E0F0D0EF93CBDFAF91EA17A1F563
:1004C600C7DF1E2FC5DF0E2FC3DF3E2FC1DF2E2F46
:1004D600A1E0B0E0E0D0E11779F4A2E0B0E0DBD033
:1004E600E01751F4A3E0B0E0D6D0E31729F4A4E076
:1004F600B0E0D1D0E21709F001C0949AA5E0B0E0CF
:10050600CAD0E11779F4A6E0B0E0C5D0E01751F4FF
:10051600A7E0B0E0C0D0E31729F4A8E0B0E0BBD074
:10052600E21709F001C0C09AC29AC49AB7DFC3D0D5
:100536002496089561DE6E2EE4E2E61509F49D9A8E
:10054600989B06C0E4E2E61511F09D9B01C001C030
:1005560004C082D0A62D9ADE8CD0EAE0E61509F416
:100566009D980895FF92AA93869903C06894F0F81F
:100576006AD072D0A0E0B0E081D0A881A13061F449
:10058600A1E0B0E07BD0A2E0B0E078D0A3E0B0E09C
:1005960075D0A4E0B0E072D06CD0AAE04ED0F0FCEA
:1005A60056D02196FF900895AA935D9BFECFE881D1
:1005B600ECB921960895BA93AA931A93E981FA8120
:1005C6003196E983FA833197E4911E2FE03019F0D2
:1005D600A12FEADFF3CFAAE0E7DF1881239608957B
:1005E600EFE1EDBDE0E0ECBD0895EFB9E1E1EDB975
:1005F600E3E1EDB9E1E1EDB9E3E1EDB9E1E1EDB951
:10060600E3E1EDB9E1E1EDB9E3E1EDB9E1E1EDB940
:10061600E3E1EDB9E1E1EDB9E3E1EDB9E1E1EDB930
:10062600E3E1EDB9E1E1EDB9E3E1EDB9EFB108954B
:10063600E1E1EDB9E3E1EDB90895B0E022C0EA9356
:10064600A4EFB1E0FBCD969AA9E3B2E80ACEA9EDF4
:10065600B2E807DE96980895C29AA0E0B0E001DEFF
:10066600C498A8EB13DEAAEA11DEADE20FDEA6ED12
:100676000DCEA0E00BDEC298C49A08950CD0AE2F22
:1006860005CE109639F086E69EE00197F1F7A8951B
:100696001197C9F70895E199FECFFF93FFB7F89434
:1006A600AEBBE09AEDB3FFBFFF9108953A932A934C
:1006B6001A930A9308953B812A8119810881089526
:00000001FF
